:1000000020210020210100001D0100001D01000031
:1000100000000000000000000000000000000000E0
:100020000000000000000000000000001D010000B2
:1000300000000000000000001D0100001D01000084
:100040001D0100001D010000890E0000350C00009C
:100050001D0100001D0100001D0100001D01000028
:100060001D0100001D0100001D0100001D01000018
:100070001D0100000000000000000000AD150000A0
:100080001D0100001D0100001D010000E519000018
:100090001D0100001D0100001D0100001D010000E8
:1000A0001D0100001D01000010B5064C2378002B37
:1000B00007D1054B002B02D0044800E000BF01230C
:1000C000237010BD38000020000000004021000017
:1000D000084B10B5002B03D00749084800E000BFCB
:1000E00007480368002B00D110BD064B002BFBD046
:1000F0009847F9E7000000003C0000204021000084
:10010000402100000000000010B5024B9847024B50
:10011000984710BD090300008D1B0000FEE700009A
:1001200010B5104A104B9A4209D00F4B0D4A03E00C
:1001300011681960043304320C498B42F8D30C4B1C
:1001400002E000221A6004330A4A9342F9D30A4AB1
:10015000FF210A4B8B439360094B9847094B984703
:10016000FEE7C046402100000000002038000020CB
:10017000380000201C01002000ED00E0000000001D
:10018000B11E0000F9190000034A516980239B0049
:100190000B4353617047C0460008004010B5034B45
:1001A000984703490348044B984710BD8901000054
:1001B00000240040B4000020B506000070B5134BC9
:1001C000DE20195C042291431954195C0125A943CE
:1001D00001242143C9B219541F38195C0F26B143B9
:1001E00002263143C9B21954DF215E5C96435E5446
:1001F0005A5CAA432243D2B25A541A5CD0390A40FC
:1002000020210A43D2B21A5470BDC046006000419A
:10021000064B4021C42299500331083A9950044AB0
:10022000D3693F390B43D3617047C046001C00407F
:100230000008004010B5044B984704490448054B9A
:100240009847054B984710BD110200000008004276
:10025000F8000020A9080000BD01000010B5024808
:10026000024B984710BDC04610E000E02D0800008A
:1002700030B50F4B5422995C0125A9430124214339
:10028000C9B299543A20195C453A9143042211436A
:10029000C9B2195455215A5CAA432243D2B25A54C6
:1002A0001A5C46390A4040210A43D2B21A5430BD82
:1002B00000600041054AD16980231B010B43D361D3
:1002C0004021E023024AD1507047C0460008004058
:1002D000001C004010B5064B9847064B9847064B4C
:1002E0009847020005490648064B984710BDC0468E
:1002F000B502000071020000D9190000002C004274
:100300009000002099090000F0B5C64600B51C4BCE
:100310009847C022D205042454601A4B1A499962A6
:100320001A49996254604220195C04252943C9B2D4
:10033000195454611C5C01218C431C549427D151E5
:10034000882691516630124C1C50C0242406A046C9
:100350001C50C024A4461C5D8C4365465C55082493
:10036000D45194510B4A1A5042461A501B301A5C11
:100370008A431A54084B984704BC9046F0BDC046C7
:100380003D0B00000060004104000240000002C07C
:1003900001000040080000405D020000830701D119
:1003A000012070470020FCE710B50C0080B2104B14
:1003B000984700280BD00C2C03D8A4000D4B1B59D8
:1003C0009F46002010E00C480EE00C480CE00C2C7E
:1003D00003D8A4000A4B1B599F46002004E009489B
:1003E00002E0064800E0084810BD0748FCE7C046A8
:1003F0009D030000F81E0000803B2600008D2700B2
:100400002C1F000000EA240080DE2800F0B5C6465C
:1004100000B50C009046866904E01F4B9C4209D34E
:10042000E41A0136B7B238001C4B98470028F4D0C4
:100430001B4BF3E70125290030001A4B98478442F3
:1004400003D3241A0135EDB2F5E70121164B9C4286
:1004500005D9164B9C4664440131C9B2F6E7002227
:10046000134B9C4205D9134B9C4664440132D2B2D3
:10047000F6E700233B2C03D93C3C0133DBB2F9E720
:100480004046C7804571017182704370047000203E
:1004900004BC9046F0BDC0468033E1019D030000DE
:1004A0000085E201A90300007F51010080AEFEFF3C
:1004B0000F0E0000F0F1FFFFF0B5DE4657464E4646
:1004C0004546E0B583B0CB880093DEB28369994698
:1004D0006A4613711379F61AF6B24F790B799A4678
:1004E0008B7898464B789B460B7801930025002427
:1004F00003E01A4B9C4664440135B5420AD24B4690
:10050000581980B2164B98470028F2D0154B9C46DC
:100510006444F1E7012505E0E9B20098124B9847E1
:1005200024180135BD42F7D35346013B0F485843C9
:100530002418E12000014346584320185B461B0164
:100540005A469B1A9C000019019B9C46604403B0CC
:100550003CBC90469946A246AB46F0BD8033E101D3
:100560009D0300000085E201A90300008051010005
:1005700070B50C00D068CD680B7C052B06D89B00AD
:100580001549CB589F46A84200D33C35E56070BD65
:10059000A842FBD3E1231B019C466544F6E7A84231
:1005A000F4D30E4B9C466544F0E7A842EED3508945
:1005B000517A0B4B98472D18E8E7A842E6D35089AB
:1005C000084B9847002803D1074B9C466544DDE75C
:1005D000064B9C466544D9E7601F0000805101002E
:1005E000A90300009D0300008033E1010085E201C2
:1005F00070B586B005000C00294B9847060001AA8B
:1006000001002800274B98470396237C052B12D81E
:100610009B00254AD3589F466B465B8963816B4696
:100620005B7A63726B461B7A23726B469B79A3716C
:100630006B465B796371261D310028001B4B984780
:10064000E0606A4621002800194B9847E1683200B3
:100650002800144B984706B070BD6B465B896381D8
:100660006B465B7A63726B461B7A23726B469B798F
:10067000A371E0E76B465B8963816B465B7A6372CB
:100680006B461B7A2372D6E76B465B8963816B46A8
:100690005B7A6372CFE76B465B896381CBE7C046C9
:1006A000550E00000D040000781F0000B904000082
:1006B0007105000070B504000D00431E9841C0B2E2
:1006C000E022520009490A4B98472368AB4208D000
:1006D000002B08D125602000064B9847064BA361EC
:1006E00070BD0020FCE712204042F9E7901F000097
:1006F000690A0000490D0000B207000010B50400AF
:10070000431E9841C0B2E622FF320449044B984789
:100710002000044B9847002010BDC046901F0000E9
:10072000690A0000D90D000030B583B004000D0047
:10073000431E9841C0B2832292000E490E4B984747
:1007400020000E4B984701006A4620000C4B98474A
:100750002B786A4613706B785370AB789370694648
:100760002000084B984701002000074B98470020C5
:1007700003B030BD901F0000690A0000550E000054
:100780000D040000B90400001D0E000030B583B058
:1007900004000D00431E9841C0B2892292000E4908
:1007A0000E4B984720000E4B984701006A462000E8
:1007B0000C4B98472B786A4613716B7853716B8892
:1007C000D38069462000084B984701002000074B62
:1007D0009847002003B030BD901F0000690A000058
:1007E000550E00000D040000B90400001D0E0000AD
:1007F00070B504000D00431E9841C0B2064A074977
:10080000074B98472000074B984701002A0020001B
:10081000054B9847002070BD3B020000901F000070
:10082000690A0000550E00000D04000010B5024BCF
:100830001860024B984710BD54000020711500004D
:1008400010B584B01438848B01AB1C801400029264
:10085000064A5A8003911900054B9847002802D197
:10086000200004B010BD0400FAE7C0460080FFFF7E
:10087000E112000010B584B01438848B01AB1C80E9
:1008800014000292064A5A8003911900054B9847BA
:10089000002802D1200004B010BD0400FAE7C046D1
:1008A0000180FFFFE112000070B504000D00431E3F
:1008B0009841C0B25E220749074B984729002000A3
:1008C000064B9847002803D1054BA361054B636194
:1008D00070BDC046AC1F0000690A00003112000064
:1008E000750800004108000010B5014B984710BD85
:1008F000611200008905890D8023DB001A400A433C
:100900008283100070471430086000207047000098
:1009100070B504000D00160000280ED000290AD082
:10092000012034220649074B9847236832002900EA
:100930002000984770BD0020F3E70020F1E7C04693
:10094000C81F0000690A000070B504000D00160001
:1009500000280ED000290AD001203D220649074B6D
:1009600098476368320029002000984770BD002036
:10097000F3E70020F1E7C046C81F0000690A000045
:1009800010B54369002B00D0984710BD10B583699E
:10099000002B00D0984710BD70B504000D00160064
:1009A000002815D0002915D0002A0FD001203322AD
:1009B00009490A4B9847E6613368290020009847A7
:1009C000074B2360074B6360002070BD0020EEE7FB
:1009D0000020ECE70020EAE7DC1F0000690A0000C5
:1009E000810900008D09000010B5041E15D0C369EF
:1009F000002B10D001204B220A490B4B9847E3698A
:100A00005B6920009847002809D1E3699B682000B2
:100A10009847002010BD0020EDE70020EBE71120F3
:100A20004042F7E7DC1F0000690A000070B50400CF
:100A30000D001600002811D0C369002B0CD0012036
:100A40007D220749074B9847E3691B69320029005B
:100A500020009847002070BD0020F1E70020EFE75C
:100A6000DC1F0000690A0000002800D100BE7047AA
:100A7000F8B505001700CE0807230B4001249C4061
:100A8000E4B200281ED0002A1ED007291ED900205B
:100A900031221449144B9847AB191B7923421ED1BC
:100AA00029001248124B9847002811D0AF60AD19A9
:100AB0002B7923432B710D4B9B191A7914431C710D
:100AC0000020F8BD0020E3E70020E1E70120DFE798
:100AD00000232B7129000548064B9847E6E70220C2
:100AE0004042EEE7F41F0000690A000058000020B1
:100AF000F90A0000110B00000368002B03D08B42A1
:100B000003D01B68F9E7002070470120FCE70000D4
:100B100070B504000D00064B984701235840C0B241
:100B200039220449044B984723682B60256070BD27
:100B3000F90A000014200000690A000010B5094BF2
:100B40005A685A600220084B9847084B9847084B50
:100B50009847084B9847084B98471F20074B9847E2
:100B600010BDC04600400041E90C0000890C0000A7
:100B7000AD0C0000790C0000E50C0000410C0000F9
:100B8000F0B583B0254B5A690192019A5A61244B02
:100B90001868431E9841C0B2DA222249224B984776
:100BA00001256D422FE0DB00204AD3185D686B1CE5
:100BB00003D01B4B1B68280098470122A240019BD1
:100BC0009343019301981A4B9847013844B2631C30
:100BD00014D00326002001E00139CEB2B042E6D89D
:100BE00033185B10D9B2FF221340DF000F4ABA5C02
:100BF000A242D8D0F0DA0131C8B2EFE7074B5A6908
:100C00000192019A5A61019B002B05D00198084B73
:100C10009847013844B2DAE703B0F0BD002800403D
:100C2000600000204C200000690A00003420000011
:100C30005D1E000010B5014B984710BD810B0000F0
:100C4000C30707D5094A0A4B1A62094B5B687D2224
:100C50001A42FAD1030707D5064A054BDA62044B5C
:100C60005B687D221A42FAD17047C0460501010037
:100C7000001C004004230100024B08229A71073A2D
:100C80001A71704700080040074A9E239382002390
:100C90009375D375D3691B0A1B02F82149010B40D8
:100CA000D3610423137470470014004082220C4B5C
:100CB0001A7538230A4AD35C9B07FAD4084BDB68C1
:100CC000DB06FBD5064A137D802149420B43DBB28C
:100CD00013753823024AD25C2A3B1A42F9D1704775
:100CE0000010004070470000094B9B78032213401E
:100CF00098420CD0064AFF239371937803218B43CB
:100D0000084018439070024B9B79002BFBD0704732
:100D10000004004010B504000268918953890B401B
:100D2000DA0502D45B0407D410BD436898472368F2
:100D3000802252009A81F7E78368984723688022CF
:100D4000D2019A81F0E7000010B5041E37D0036885
:100D5000002B32D001202F221A491B4B98471B4BE6
:100D60001C6021680A691A4B1A42FBD10B889B0749
:100D70000BD50B88022293430B800A69144B1A424D
:100D8000FBD1226813699B07FCD4226813880121D8
:100D90000B439BB213801369DB07FCD423681A69E9
:100DA000D207FCD40B4A1A801969094A1142FBD1B7
:100DB000236800221A66002010BD0020CBE7002027
:100DC000C9E7C04664200000690A000064000020F2
:100DD00003800000008BFFFF10B5041E15D00368D0
:100DE000002B10D00120732209490A4B9847216833
:100DF0000B88022213439BB20B800A69064B1A42EE
:100E0000FBD1002010BD0020EDE70020EBE7C0463D
:100E100064200000690A00000380000070B504002F
:100E20000D00002810D00368002B0BD001208B226E
:100E30000649074B98472268956113691B07FCD444
:100E4000002070BD0020F2E70020F0E764200000E1
:100E5000690A000010B5041E0FD00368002B0AD0E9
:100E6000012097220649074B9847226813691B0700
:100E7000FCD4906910BD0020F3E70020F1E7C046E4
:100E800064200000690A000010B5024B1868024B8C
:100E9000984710BD64000020150D0000024B9C46D1
:100EA0006044800AC0B2704700FCFFBD10B50D4B16
:100EB00098470023002B08D0E62292000A49002020
:100EC0000A4B98470120404210BD5A00D218D10069
:100ED000074A5218127D904202D00133DBB2E9E793
:100EE00058B2F1E79D0E0000CC200000690A000016
:100EF0007C20000070B505000C0008002D4B9847C1
:100F0000C0B2E369DB071DD443001B18DA002A4B8B
:100F10009B189A691C231A40E3699B07FCD123683C
:100F20009B0709D5236802218B432360E3699B0754
:100F3000FCD1E3699B07FCD4012313432360E369DD
:100F40009B07FCD1E369DB07FCD443001B18DA00E4
:100F5000194B9B189B692360E3699B07FCD14300F5
:100F60001B18DA00144B9B18DB696360E3695B07AD
:100F7000FCD442001218D1000F4B5B181A6AE260D1
:100F8000DA7E03231A40AA81023B93429B415B42D3
:100F9000626A0A490A409B0313436362E3695B0781
:100FA000FCD443001818C200034B9B18DB8CEB8168
:100FB000002070BDAD0E00007C200000FFBFFFFFD1
:100FC00070B5050004692368DB0E01261E40431E30
:100FD0009841C0B28E4A8F498F4B98476B68012B5E
:100FE0004DD063688D4A13406360E3695B07FCD4AE
:100FF0002B885A054ED56A88D20704D56A88802185
:10100000C9000A436A805B00854A1A40E3695B07AE
:10101000FCD4636A8021C9010B4013438022120271
:1010200013436362E3695B07FCD42E697D4A337E18
:10103000DBB21800511E002A02D00A009B07F6D02E
:101040002368DB0E01221A40E3695B07FCD4638B43
:101050009BB2C10700D48FE09A072FD501222276D8
:101060006A88802149010A436A806A886E490A4079
:101070006A80DB0700D4C6E005204042A2E0002ED3
:10108000AFD062688023DB0213436360E3695B07D0
:10109000FCD4ADE75B00FF2213406A8801210A40BF
:1010A0001A43E3695B07FCD4636A8021C9010B40E2
:1010B00013436362E3695B07FCD4B6E75B071BD4A9
:1010C0006B885B0534D52A881212520006231A4019
:1010D000E3695B07FCD4636A8021C9010B401343B9
:1010E000F12213436362E3695B07FCD46B884F4AC8
:1010F00013406B80002065E06B68002B04DD6B887B
:101100008022520113436B806B881BB2002B06DBDD
:101110006B88454A13406B800220404252E062686F
:10112000C0239B0213436360E3695B07FCD4EFE7D2
:101130006868002811D16B881BB2002B04DB6B8818
:10114000394A13406B803DE06268C0239B02134321
:101150006360E3695B07FCD4F1E7AB681A78282386
:10116000E254E3695B07FCD4AB680133AB606B68A6
:10117000013B6B60002025E0810747D569680029A5
:101180003CD05B073AD401396960002901D1002ABB
:101190001BD0012917D06B68002B07D16B881BB2BD
:1011A000002B1BDB6B88204A13406B80AA68531C02
:1011B000AB60E3695B07FCD42823E35C1370022374
:1011C0002376002070BD002AE5D062688023DB0210
:1011D00013436360E3695B07FCD4DCE76368124A8E
:1011E00013406360E3695B07FCD46268C0239B0221
:1011F00013436360E3695B07FCD4D3E702232376E0
:1012000002204042DEE704204042DBE70020D9E72D
:1012100094050000CC200000690A0000FFFFFBFFDE
:10122000FE070000FFFF0000FFFEFFFFFFFBFFFFC8
:1012300070B504000D00431E9841C0B2044A054930
:10124000054B9847256129002000044B984770BD45
:1012500007050000CC200000690A0000F50E000020
:1012600070B50400194D431E9841C0B2184A2900B8
:10127000184EB04724692000431E9841C0B2164A58
:101280002900B0472368022213432360E3699B07C8
:10129000FCD104201149E3695B07FCD4628B12097D
:1012A00003231340012B0BD001390029F3DC013853
:1012B000002807D010236383E3695B07FCD4E9E7C8
:1012C000002070BD06204042FBE7C046CC20000055
:1012D00024050000690A0000F4050000FFFF00007B
:1012E000F8B505000E000469431E9841C0B2934A48
:1012F0009349944FB8472869431E9841C0B2B82219
:10130000D2008F49B8473000431E9841C0B28E4A80
:101310008B49B8476B88DB0500D50BE172888023C9
:101320005B009C461A4372802A00310089C989C239
:101330006268634613436360E3695B07FCD428007B
:10134000824B9847002800D19DE06B88804A13406B
:101350006B80F8BD05204042A6E073881BB2002BCD
:1013600004DB6B887A4A13406B80F2E76268C02323
:101370009B0213436360E3695B07FCD4F1E7530707
:101380001BD46B885B0534D52A88121252000623C1
:101390001A40E3695B07FCD4636A8021C9010B40F2
:1013A0001343F12213436362E3695B07FCD46B8848
:1013B000684A13406B80002065E06B68002B04DDF9
:1013C0006B888022520113436B806B881BB2002B09
:1013D00006DB6B885E4A13406B800220404252E07D
:1013E0006268C0239B0213436360E3695B07FCD41C
:1013F000EFE76868002811D16B881BB2002B04DB73
:101400006B88534A13406B803DE06268C0239B02A7
:1014100013436360E3695B07FCD4F1E7AB681A78B8
:101420002823E254E3695B07FCD4AB680133AB606B
:101430006B68013B6B60002025E0BB0778D56B68CB
:10144000002B6DD052076BD4013B6B60002B01D198
:1014500000294CD0012B48D06B68002B07D16B883A
:101460001BB2002B4CDB6B88394A13406B80AA6897
:10147000531CAB60E3695B07FCD42823E35C137067
:101480000223237600206B88DB0500D461E72869FE
:10149000314A037EDBB21F00511E002A00D159E7FA
:1014A0000A009B07F5D00020002800D055E72368EC
:1014B000DB0E01211940E3695B07FCD4628B92B219
:1014C000FB07BAD5930700D459E7012323766B882D
:1014D000802149010B436B806B881D490B406B8059
:1014E000D30722D505204042CDE70029B4D0626859
:1014F0008023DB0213436360E3695B07FCD4ABE743
:101500006368134A13406360E3695B07FCD4626855
:10151000C0239B0213436360E3695B07FCD4A2E72B
:101520000223237602204042ADE704204042AAE78E
:101530000020A8E7062040420BE7C046BF05000098
:10154000CC200000690A0000C1050000C10F0000A6
:10155000FFFEFFFFFFFBFFFFFFFF0000024B034A00
:101560005A6005221A60704710E000E0FFFFFF009C
:1015700010B5014B984710BD5D15000070B5050012
:101580000469E36ADB0705D50123E3620368002BE6
:1015900000D09847A36A1B0706D50823E3626B684F
:1015A000002B01D02800984770BD000010B5024BF9
:1015B0001868024B984710BD680000207D15000098
:1015C0000269136802210B43136013699B07FCD166
:1015D00070470269136802218B43136013699B07EC
:1015E000FCD17047026913699B07FCD113685B0843
:1015F00001201840704770B505000469A37ADB0725
:1016000005D50123A3720368002B00D09847637AA5
:101610009B0706D50223A3726B68002B01D028001C
:10162000984770BD034B984200D07047024B196039
:10163000FBE7C046002C00426C00002010B50E4BAA
:101640009C466044800AC3B20020002808D0B02223
:1016500052000A4900200A4B98470120404210BD21
:10166000820012189100074A8A5C9A4202D0013027
:10167000C0B2EAE740B2F2E700E0FFBDE8200000B8
:10168000690A00000000002070B506000C00080088
:10169000534B9847050034612369DB0714D4236951
:1016A0009B07FCD123689B0709D52368022293433B
:1016B000236023699B07FCD123699B07FCD401238A
:1016C000236023699B07FCD12369DB07FCD4AB00B3
:1016D0005B199A00434B9B185B68236023699B0747
:1016E000FCD1AA00521991003E4B5B189A7AE27322
:1016F0001A89E280032222735A680C231340082BB4
:1017000054D0002B66D1AB005B199A00354B9B1867
:101710009B89A3832369C0221A42FBD1AB005B19CA
:101720009A00304B9B181B8AE3832369C0221A421C
:10173000FBD1310020002C4B9847AB005B199A007D
:10174000284B9B185B785BB2002B0BDB1F221340EE
:101750001E3A9A401300802224498B50BFF34F8FCA
:10176000BFF36F8FAB005B199A001E4B9B185B7821
:101770005BB2002B08DB1F2213401E3A9A40130075
:10178000C022520019498B50AB005D19AA00154BBD
:101790009B185B785BB2002B1FDB1F2213401E3AA5
:1017A0009A401300114A1360002070BD0D4B5B1866
:1017B000DB68E3612369C0221A42FBD1AB005B19ED
:1017C0009A00084B9B181B6923622369C0221A42A6
:1017D000FBD1AEE701204042E7E70020E5E7C04645
:1017E0003D160000000000202516000000E100E08A
:1017F00070B50E001500046920001B4B984782004D
:1018000012189100194B5B18DE601D615A680C2399
:101810001340082B16D083001B189A00134B9B18FB
:101820009B89A3832369C0221A42FBD18300181825
:1018300082000E4B9B181B8AE3832369C0221A4245
:10184000FBD170BDE6612369C0221A42FBD183003F
:1018500018188200054B9B181B6923622369C0225C
:101860001A42FBD1EDE7C0463D1600000000002003
:1018700010B5046920000C4B9847830018188200AB
:101880000A4B9B185A680C231340082B06D0236977
:10189000C0221A42FBD1A08B80B210BD2369C022A6
:1018A0001A42FBD1E069F8E73D1600000000002075
:1018B00010B504692000144B984783001818820063
:1018C000124B9B185A680C231340082B11D0236924
:1018D000C0221A42FBD1A18B89B22369C0221A42CD
:1018E000FBD1E38B9BB2FA2080005843084B98470A
:1018F00010BD2369C0221A42FBD1E1692369C022CD
:101900001A42FBD1236AEEE73D16000000000020DA
:10191000451D000070B504692000164B984705006E
:10192000C22215490120154B9847A8004019820092
:10193000134B9B185B785BB2002B0BDB1F22134011
:101940001E3A9A40130080220E498B50BFF34F8FEE
:10195000BFF36F8F236802229343236023699B07A1
:10196000FCD123680122134323602369DB07FCD4E5
:1019700070BDC0463D160000E8200000690A000066
:101980000000002000E100E070B504000E0015002A
:10199000431E9841C0B21822FF320D490D4B9847A3
:1019A000002E08D12369002D02D101221A7204E011
:1019B00001225A7201E0012E00D070BD2369002D72
:1019C00002D002225A72F8E702221A72F5E7C046E4
:1019D000E8200000690A0000014814307047C04642
:1019E0000000002010B5024B1868024B984710BD4C
:1019F0006C000020F715000030B58BB0234B9847E2
:101A000002AC234BE3800423637119222271A3707B
:101A100000256570257004A81E4B98471E4B9847FB
:101A20001E4B9847029861681D4B984724201D4B18
:101A3000984710219823C022D205D1501A4B9847BD
:101A40006B46DC1DDD71991DD0230B7001227720C0
:101A5000164B9847012221007720154B9847237891
:101A6000602B01D1134B984702AB1C7801E0114B5E
:101A70009847250002AC20000F4B98472478A542D8
:101A8000F8D0E307F3D40D4B9847F2E709010000C3
:101A9000E5070000B11B0000B51B0000191C000089
:101AA000351C0000751C0000B91C0000E51C00007E
:101AB000151D0000051C0000611C0000F11B00004A
:101AC00070B582B00E00002813D1164B1D680CE0D3
:101AD000737801AC63700123237020006B68984712
:101AE00032782378134033702D68002DF0D102B086
:101AF00070BD022804D00128F9D10A4B9C680DE082
:101B0000084B5C6803E0F0B2636898472468002CD7
:101B1000F9D1ECE7F0B2636898472468002CF9D15A
:101B2000E5E7C0467000002070B5084E084C0C3444
:101B3000320001212000074DA8473200002120007B
:101B4000A847320002212000A84770BDC11A00003A
:101B500070000020710A000010B50400431E984177
:101B6000C0B240220349044B984721000348044B6C
:101B7000984710BDFC200000690A0000700000209A
:101B8000110B0000002303707047000010B5044BD8
:101B900098470448044B4360044B984710BDC04627
:101BA000291B000088000020851B0000591B000035
:101BB0007047000010B5064B9847064C00220649B6
:101BC0002000064B98472000054B984710BDC046A3
:101BD000D502000090000020102700002D0A000010
:101BE000E9090000014B9883D9837047002C00421B
:101BF00010B500210148024B984710BDFFFF0000BF
:101C0000E51B000010B502490020024B984710BDAB
:101C1000FFFF0000E51B000010B5034B9847034889
:101C2000034B984710BDC0469D010000B400002042
:101C3000FD06000010B582B000900191054C01A98D
:101C40002000054B984769462000044B984702B096
:101C500010BDC046B40000208D0700002907000019
:101C600010B501000148024B984710BDB400002098
:101C7000F107000070B543091F2404400125290025
:101C8000A140DA01C020C005101881600E04360C96
:101C90008020C0053043074EB44662449062090C70
:101CA000C020000601439162101940300378AB4315
:101CB000037070BD0060004110B5054B9847054C9E
:101CC00005492000054B98472000054B984710BD5B
:101CD00035020000F800002018010020070900006C
:101CE000E908000070B50C00150080221201010007
:101CF0000448054B9847054B18682A002100044BFF
:101D0000984770BDF8000020F50800001801002079
:101D10001109000070B50C001500802212010100AD
:101D20000448054B9847054B18682A002100044BCE
:101D3000984770BDF8000020F50800001801002049
:101D400049090000002243088B4274D303098B42E7
:101D50005FD3030A8B4244D3030B8B4228D3030C7B
:101D60008B420DD3FF22090212BA030C8B4202D31D
:101D70001212090265D0030B8B4219D300E0090A45
:101D8000C30B8B4201D3CB03C01A5241830B8B424E
:101D900001D38B03C01A5241430B8B4201D34B0337
:101DA000C01A5241030B8B4201D30B03C01A52419C
:101DB000C30A8B4201D3CB02C01A5241830A8B4221
:101DC00001D38B02C01A5241430A8B4201D34B020A
:101DD000C01A5241030A8B4201D30B02C01A52416E
:101DE000CDD2C3098B4201D3CB01C01A5241830922
:101DF0008B4201D38B01C01A524143098B4201D35C
:101E00004B01C01A524103098B4201D30B01C01A86
:101E10005241C3088B4201D3CB00C01A5241830800
:101E20008B4201D38B00C01A524143088B4201D32D
:101E30004B00C01A5241411A00D20146524110468D
:101E40007047FFE701B5002000F006F802BDC0466C
:101E50000029F7D076E770477047C04610B50023D9
:101E6000002802D000F004F8431C180010BDC04642
:101E7000414208401C2101231B04984201D3000C5D
:101E800010391B0A984201D3000A08391B099842ED
:101E900001D30009043902A2105C401A7047C04601
:101EA0001B1C1D1D1E1E1E1E1F1F1F1F1F1F1F1F51
:101EB00070B500260C4D0D4C641BA410A64209D130
:101EC000002600F02DF90A4D0A4C641BA410A6420E
:101ED00005D170BDB300EB5898470136EEE7B3006B
:101EE000EB5898470136F2E72C2100002C21000026
:101EF0002C21000030210000C2030000E603000096
:101F0000C6030000E6030000CA030000E603000069
:101F1000CA030000E6030000E6030000CA03000055
:101F2000E6030000CA030000E6030000DA03000035
:101F3000EA030000DE030000EA030000E203000001
:101F4000EA030000E2030000EA030000EA030000E5
:101F5000E2030000EA030000E2030000EA030000DD
:101F60008C05000086050000900500009E0500001D
:101F7000AA050000BA050000360600001806000099
:101F80005A0600007406000088060000960600004D
:101F90002E2E2F68616C2F7372632F68616C5F63E4
:101FA000616C656E6461722E630000002E2E2F68D6
:101FB000616C2F7372632F68616C5F6932635F6D50
:101FC0005F73796E632E63002E2E2F68616C2F7302
:101FD00072632F68616C5F696F2E63002E2E2F680D
:101FE000616C2F7372632F68616C5F70776D2E6305
:101FF000000000002E2E2F68616C2F7574696C73C1
:102000002F7372632F7574696C735F6576656E7478
:102010002E6300002E2E2F68616C2F7574696C730F
:102020002F7372632F7574696C735F6C6973742E90
:10203000630000000500000025000000060000000D
:102040001600000007000000170000002E2E2F6869
:10205000706C2F6569632F68706C5F6569632E63B0
:10206000000000002E2E2F68706C2F7274632F6892
:10207000706C5F7274632E6300000000000000004B
:102080000000000000000000000000000000000050
:102090000100000014002000000100000E0F0000ED
:1020A0000000D70000093D00000000000000000013
:1020B0000000000000000000000000000000000020
:1020C0000000000000000000000000002E2E2F681D
:1020D000706C2F736572636F6D2F68706C5F7365C2
:1020E00072636F6D2E6300002E2E2F68706C2F743C
:1020F000632F68706C5F74632E6300002E2E2F7345
:102100006C6565705F6D616E616765722F736C657C
:1021100065705F6D616E616765722E63000000001F
:10212000F8B5C046F8BC08BC9E467047D100000018
:10213000F8B5C046F8BC08BC9E467047A900000030
:102140000313000000000000000000329F0F000099
:10215000CF0700008916000015190000C115000006
:10216000D3150000F1170000E515000071180000FC
:08217000B118000089190000FC
:00000001FF
